:020000040800F2
:100000000002002071040008C5040008D50400089F
:10001000E5040008F50400080505000800000000DC
:100020000000000000000000000000000D040008B7
:100030001505000800000000F10300080B0200088D
:100040000B0200080B0200080B0200080B0200085C
:100050000B0200080B020008E90D0008E90D00087A
:10006000E90D0008E90D0008E90D00080B02000881
:100070000B0200080B020008F50B00080B02000839
:100080000B020008BD0B00080B0200080B02000861
:100090000B0200080B0200080B020008E90D000823
:1000A0000B0200080B0200080B0200080B020008FC
:1000B0000B0200080B0200080B0200080B020008EC
:1000C0000B0200080B0200080B020008E5180008EC
:1000D000F11800080B020008B10B0008E90B00083A
:1000E000E90D00080B0200080B0200080B020008D3
:1000F0000B0200080B0200080B0200080B020008AC
:100100000B0200080B0200080B0200080B0200089B
:100110000B0200080B0200080B0200080B0200088B
:100120000B0200080B0200080B0200080B0200087B
:100130000B0200080B0200080B0200080B0200086B
:100140000B0200080B0200080B0200080B0200085B
:100150000B0200080B0200080B0200080B0200084B
:100160000B0200080B0200080B0200080B0200083B
:100170000B0200080B0200080B0200080B0200082B
:100180000B0200080B02000800F0D4B97047000011
:1001900070B50C46064600F059F9094B094A1D682E
:1001A0002919914202D8084A914204D20C233360A3
:1001B0004FF0FF3500E0196000F050F9284670BD9F
:1001C0000002002000000220FC0E0020194610460C
:1001D00000F0BCB91946104600F0C0B91323036003
:1001E0004FF0FF307047132303604FF0FF3070472C
:1001F000132303604FF0FF30704702294FF00003D4
:1002000003608CBF00200120704700F08BB9000014
:10021000114B70B500241C60104B114D18682E68EE
:1002200000F09CF80F4B53F820301B68A3F1080234
:1002300096420FD026B13179092904BF0A213171C4
:10024000092103F8041C33F9021C074B2A601980AA
:10025000012070BD204670BD18040020EC04002071
:1002600020040020280400201C040020082930B5A8
:10027000037919D9082B32D842791A4B53F82250F6
:1002800000F108042DB12D68856053F822502C60D0
:1002900000E0846043F82240134C4279012303FAC2
:1002A00002F22368134319E0082B18D945790D4B46
:1002B00053F825203AB11468A2420BBF00222468EB
:1002C00043F825201460427953F822303BB9064C9C
:1002D000012303FA02F2236823EA02032360017177
:1002E00030BD00BF28040020EC04002008B50A4BF4
:1002F0001B681A79082A02D95B7983420AD900F06F
:10030000B0F818B1054B01221A6008BDBDE80840DD
:1003100000F066B808BD00BF2004002018040020CB
:1003200008B500F093F8094B094A1B88094D1BB228
:10033000002442F82340084A286813682146013BFC
:100340001360FFF793FF2C6000F046F81C040020B8
:100350006804002020040020240400200023C20799
:1003600002D440080133FAE718467047134423F0DB
:10037000030310B54FF077321C1F43F8042C6207BB
:1003800042BF4FF0883243F8082CA3F108044FF025
:10039000807304E909000F4B44F80C3C002344F837
:1003A000103C032344F8143C2246022344F8183C32
:1003B000012344F81C3C42F8201D0B2342F8043D65
:1003C000013B032BFAD120466FF0020340F8443D75
:1003D00010BD00BF2103000800F03CF801DFFEE77C
:1003E000024A536843F080535360704700ED00E0C9
:1003F000EFF3098020E9F00F40F804ED02490968A5
:10040000086000F003F8000020040020FFF700FF60
:1004100004480068016801C9B1E8F00F81F3098858
:100420000047000020040020BFF34F8F0549064B12
:10043000CA6802F4E0621343CB60BFF34F8F00BF82
:10044000FDE700BF00ED00E00400FA05EFF31080C7
:1004500072B6704762B6EFF31080704780F3108871
:100460007047EFF30580C0B27047704770470000D7
:1004700008B5FFF7FAFF0E4A0E4B0F498B4204D224
:1004800052F8040F43F8040BF8E70C4B0C4A002118
:10049000934202D243F8041BFAE7FFF7E7FF00F0AC
:1004A00067F801F0D7FFBDE8084000F0ADB800BF25
:1004B000AC3E0008000200201804002018040020B0
:1004C000FC0E002008B50249042000F06FF800BFC0
:1004D0005033000808B50249052000F067F800BF56
:1004E0005C33000808B50249062000F05FF800BF41
:1004F0006F33000808B50249072000F057F800BF25
:100500008233000808B50249082000F04FF800BF08
:100510009433000808B50249092000F047F800BFED
:10052000A833000808B502490A2000F03FF800BFD0
:10053000BA330008034B044A4FF4E131002000F0C5
:1005400071BA00BF04020020F50800080A460146FF
:10055000014800F0DAB900BF0402002010B50A46D5
:100560000C460146002000F007FA204610BD0000AE
:1005700008B50121094800F053FB0121084800F0AB
:100580004FFB0121074800F04BFB0121064800F01A
:1005900047FBBDE8084000F0F7B800BF0D0C024073
:1005A0000C0C02400E0C02400F0C024008B5084B28
:1005B0001A683AB9012207481A6002F025F806487D
:1005C00002F022F8FFF742FF00F0DCF8FFF72CFF03
:1005D00030050020C8330008E433000808B500F0F7
:1005E00055FF034802F010F800F038FF002008BD66
:1005F000F733000808B5034C2368012000F044F9E4
:10060000FAE700BF340C00201FB5FFF71FFF0E4BA9
:100610000E481B68029300240D4B00930F220C23FD
:100620004FF48071019400F045F80A4B0A481B68AA
:1006300002930A4B009307220C234FF4C0610194EC
:1006400000F038F8FFF7C8FE18020020340500203B
:10065000F50500081C02002034060020DD05000816
:1006600008B5FFF7F3FE094B1B681A79082A07D96A
:100670005A79074B53F8221011B1096843F8221038
:10068000FFF7ECFEBDE80840FFF7AABE20040020FB
:100690002804002030B54C7901F1080203682BB121
:1006A00013F8035CAC4201D31846F7E78B60026095
:1006B00030BD00000F2A2DE9F84F804691469A463A
:1006C00020D810F003031CBFC3F10403C91AA1F121
:1006D000240118BF984421F00307FFF7B7FE274A0B
:1006E00008EB07048346012352F823601DB26EB164
:1006F0000133212BF8D15846FFF7B0FE6FF08A0086
:10070000BDE8F88F6FF01500BDE8F88F1B4A0B9914
:1007100042F823400A98E5803B464246FFF726FE12
:10072000174A20604FF0FF33E361136884F80590A7
:1007300001331AF0010F2671A660E660266166613A
:10074000A6612662136004D001212046FFF78EFDCA
:100750000DE00A212046FFF789FD1AF0040F06D1AB
:100760005846FFF77BFE4846FFF7C0FD02E05846BB
:10077000FFF774FE2846BDE8F88F00BF680400202C
:10078000240400207047000010B500F0D7FE3B4B5A
:10079000002199601A6822F0867222F480321A6071
:1007A000D9601A6842F480321A601A68334C900398
:1007B000FBD54FF08051002000F03EFB304A13681B
:1007C00043F400431360A36823F0F003A360A3681D
:1007D000A360A36823F46043A360A36843F40043C9
:1007E000A360A36823F4E053A360A36843F4A05379
:1007F000A36000236360636843F4800363606368FD
:1008000043F008036360636843F4A843636063686C
:100810006360636843F0E0636360236843F0807360
:1008200023602368154A9901FBD5164B00211960F6
:10083000196841F400711960196841F48061196008
:10084000196821F00F011960196841F0050119605C
:10085000936823F003039360936843F0020393606B
:10086000936813F0080F054BFAD01A6822F00102C2
:100870001A601A689207FCD410BD00BF003802400D
:1008800000700040003C0240174B93F90010042810
:1008900027D8DFE800F003060D15150000221A70B6
:1008A0001FE001221A70114A136923F0040316E0B5
:1008B00002221A700E4A136823F0030313600AE041
:1008C00003221A700A4B1A6842F00E021A605A6824
:1008D00042F480725A60054A136943F004031361BD
:1008E00030BF0846704700BF2002002000ED00E046
:1008F0000070004038B50446043000F0D6FA0546D2
:10090000204600F0F5FD284638BDF8B504460E46F1
:100910001746051D3A463146284600F0B1FA20B97F
:100920000121204600F0B4FDF4E7F8BD420901239F
:1009300000F01F0003FA00F0014B43F8220070475B
:1009400000E100E008B50B689B0608D5084B496834
:1009500003EBC002C9B253F8303050689847054BDA
:100960001B681BB1BDE80840FFF77ABE08BD00BF99
:10097000480C0020180400202DE9F84306460C46D8
:100980001546FFF76EFDDFF8849078B118237343A6
:10099000254459F80330AC4206D01A681206FCD53B
:1009A00014F8012B5A60F6E7BDE8F883134F4FEABD
:1009B000860847440121384600F06AFD182202FBF0
:1009C00006960F48F37C0F49072BC8BF014610203D
:1009D00003F0070312FB0303CA18ADB2D4605560DD
:1009E000CA58094842F00102CA504044012100F0AF
:1009F0004FFD3846BDE8F84300F07ABD380C0020C2
:100A00000064024000600240400C002044340008B2
:100A1000034A182303FB00204168407C00F00CBA15
:100A20004434000801282DE9F84F05460C4600F231
:100A3000A88018214143554F07EB01087E585449BF
:100A400041F8302001EBC0014FF000094B60514BE1
:100A500043F820905048012140F8259000EB850094
:100A600000F016FDD8F808B04946584600F0D8F80E
:100A7000D8F80C900121484600F0D2F898F810A060
:100A80005846514600F074F95146484600F070F956
:100A90002846FFF7BDFF98F8113021010BB93F48F8
:100AA00000E03F48B0FBF1F001F05EF9804601F054
:100AB00003FB84B2204601F05BF90146404601F099
:100AC000A1F84FF0834101F0A7F901F0F5FA2401F4
:100AD000A4B200F00F0020438023B06073610023B4
:100AE000336142F20C03F360182303FB0573DC7CD3
:100AF000072C06DC4FF40011022000F09DF9294973
:100B000005E04FF48001022000F096F9264904F038
:100B100007031820102210FB032200FB057001EBD5
:100B2000020E037D90F912005B0643F4823343F01A
:100B300050038B50331DCEF808300023CEF814300C
:100B4000FFF7F4FE062C02DC04F10B000FE0072C8B
:100B500004D1164B4FF400425A600BE00C2C02DC1F
:100B600004F1300003E00F2C04DC04F1370040B244
:100B7000FFF7DCFEF36843F02003F3600020BDE8DC
:100B8000F88F4FF0FF30BDE8F88F00BF4434000805
:100B9000480C0020380C0020400C002080DE800231
:100BA00000BD0105006002400064024000E100E079
:100BB00001490020FFF7C6BE0044004008B5074BBE
:100BC00007484FF40012DA6000F092FC054B1B68F6
:100BD0001BB1BDE80840FFF743BD08BD00600240FF
:100BE000400C00201804002001490120FFF7AABE94
:100BF0000048004008B5074B07484FF000629A6074
:100C000000F076FC054B1B681BB1BDE80840FFF700
:100C100027BD08BD00600240440C002018040020DD
:100C2000F8B50E460125C0F3832120F00F0400F033
:100C30000F0705FA01F1022000F0FEF807FA05F0AF
:100C40000323216883406FEA030C01EA0C01216051
:100C5000216806F0030E0EFA00FE4EEA0101216043
:100C6000E2680CEA0202E260E168C6F381028240B7
:100C70000A43E2606268BD4022EA0502626062687F
:100C8000C6F30016BE4016436660A268ADB21343B9
:100C9000A36000206583F8BD2DE9F04100F00F044A
:100CA0001646304A42F8343002EBC402069B5360C9
:100CB00005468846C0F383274FF48041012000F0A9
:100CC000BBF841462846FFF7ABFF042C264B03DC5C
:100CD000A11D01228A4003E0092C03DC4FF400022D
:100CE0001A6002E04FF480725A60012E1F4B07D049
:100CF0000FD3022E16D199680122A24011430DE0B4
:100D00009A68A64032439A60DA6822EA0606DE60F4
:100D100008E099680122A24021EA02019960D9689D
:100D20000A43DA6004F00C0303F1804303F59C33BB
:100D300005F003059968AD000F22AA4021EA0202DE
:100D40009A609A6807FA05F515439D60012303FA36
:100D500004F4064B5C611A6814431C600020BDE873
:100D6000F08100BF580C002000E100E0003C014091
:100D700020F00F0300F00F02F0B51E6857000325A6
:100D8000BD4026EA05051D601D680224072A04FAF5
:100D900007F444EA050494BF002201221C6003EB1F
:100DA000820300F007001C6A80000F22824024EAC0
:100DB00002021A621A6A814041EA02001862F0BD1A
:100DC00020F00F02012300F00F0003FA00F080B2C0
:100DD0001083704720F00F02012300F00F0003FA88
:100DE00000F080B250837047104B2DE9F0415E69EE
:100DF0001A680F4F164000244FF001081D4608FAEC
:100E000004F31E4206D06B6107EBC40357F834208D
:100E1000586890470134102CF1D1064B1B681BB168
:100E2000BDE8F041FFF71CBCBDE8F081003C01408B
:100E3000580C00201804002004281CD8DFE800F01B
:100E400003080D1217000D4B1A6C1143196412E0C0
:100E50000A4A536C194351640DE0084A136B194355
:100E6000116308E0054A536B1943516303E0034AD9
:100E7000936B19439163BFF34F8F70470038024063
:100E800070B513467BB18568C468A5420BD08468F1
:100E90000668651C85604568013D2C40013B345D5A
:100EA00001F8014BEEE7D01A70BDC368426830B557
:100EB00084681B1B934208D0C3680468013A5D1C18
:100EC0001340C560E154002030BD4FF0FF3030BD0D
:100ED00008B5064B4621187800F0F6FC044B0022BA
:100EE0001A60044B02221A7008BD00BF44020020A1
:100EF000E00C0020D80C00201B4A1C491368C85481
:100F00000133FF2BC8BF00231360194A1378012B4C
:100F100009D002D3022B0CD023E0164A1368591CC7
:100F20001160154A0EE0134A1368013313606F20F5
:100F3000704720280F4B07D1002111701A68511CEF
:100F400019600D4BD05C7047010606D5012100F0F9
:100F50007F001860117057207047002111701860D1
:100F6000ECE76520704700BFDC0C0020E40D00209A
:100F7000D80C0020E00C0020743400082DE9F84360
:100F8000DFF8C091564E574C4FF00008022303285B
:100F900007460D46C9F8008086F8008023703BDCC8
:100FA0000968514801F030FB504801F09FFB424670
:100FB00041464F4801F028FB012211464C4801F000
:100FC00023FB4C4801F092FB4B4801F08FFB4B4850
:100FD00001F08CFB4A4801F089FB4A4801F086FB8E
:100FE000494801F083FB494801F080FB484801F083
:100FF0007DFB484801F07AFB474801F077FB474802
:1010000001F074FB464801F071FB464801F06EFBAD
:101010006FF00300BDE8F883486801F06DF801281F
:10102000C9F8000006D9404801F060FB4FF0FF30DE
:10103000BDE8F883A868DFF8108101F05DF8C8F812
:101040000000E86801F058F8384B1860D8F8003014
:101050009B0203F1804303F500331843344B042F04
:1010600018603AD02B69334A1B78303B032B13604E
:1010700006D9314801F03AFB6FF00100BDE8F88372
:10108000022B04D0032B02D0012B18BF0023052F05
:10109000337022D06B6929491B78A3F13002042AEE
:1010A0000A6006D9264801F021FB6FF00200BDE876
:1010B000F883313B032B03D8DFE803F007090B0D5E
:1010C000002323701846BDE8F883012304E00223BF
:1010D00002E0032300E0042323700020BDE8F8832E
:1010E0002C0200203C020020C3340008F634000823
:1010F0001C350008363500086C350008A535000899
:10110000F1350008283600086036000898360008D7
:10111000D1360008213700083A3700085337000855
:101120006A370008813700089A3700082802002033
:101130002402002034020020B937000840020020B9
:10114000D937000844020020380200202DE9F3417D
:10115000234F4FF0FF333B60FFF710FF00283BDBCE
:10116000204C207800F076FB1F4B20781A781F4B1C
:10117000197800F0A3FA0546207800F07BFB002DDB
:1011800005DA2A4621681A4801F03EFA24E0DFF821
:101190007C80184ED8F80000174D0121FFF740FD64
:1011A000031E05DA32682968144801F02DFA13E0AD
:1011B000D8F80000FFF704FE01233B60104B2168C4
:1011C0001B6801930F4B10481B6800932A68336813
:1011D00001F01AFA002000E0012002B0BDE8F08121
:1011E00030020020440200203C0200202C0200209B
:1011F000FA3700082802002038020020373800089B
:1012000040020020340200207C3800082402002024
:1012100073B5204E4FF0FF333360FFF7AFFE002869
:1012200034DB1D4D287800F015FB1C4B1C4A197847
:10123000287800F0AFFA0446287800F01BFB002C59
:1012400005DA22462968174801F0DEF91EE000247D
:1012500015480094154B006822462146FFF71CFDF7
:10126000031E134A134905DA12680968124801F08F
:10127000CBF90BE0114B12481B68009313680A6806
:101280002968346001F0C0F9204600E0012002B076
:1012900070BD00BF30020020440200202C0200205C
:1012A000F90E0008D238000824020020D10E0008F0
:1012B00028020020380200200F39000834020020E4
:1012C0005839000870B50C4601461A48164601F018
:1012D0009BF90025B54205DA2946174801F094F933
:1012E0000135F7E7154801F08FF925462B1B9E4283
:1012F00005DD15F8011B124801F086F9F6E70F48E5
:1013000001F082F925462B1B9E420DDD15F8011BCD
:10131000A1F120035E2B03D90A4801F075F9F2E729
:10132000094801F071F9EEE70848BDE8704001F0A6
:101330006BB900BFA2390008A6390008AD39000812
:10134000B3390008BB390008C1390008F43300087C
:10135000234B2DE9F0411D68012D04D0214801F0F7
:10136000C5F9012538E0012804DC1F481F4E01F0B3
:10137000BDF900E04E681E4FDFF88C80387800F031
:1013800069FAD8F80000FFF725FD30463C7801F0F7
:101390002EFA31460346174A204600F0AFFA0446BB
:1013A000D8F80000FFF70CFD387800F063FA002C45
:1013B000214603DA104801F027F90DE00F4801F04B
:1013C00023F9224631460E48FFF77CFF22460949A1
:1013D0000C48FFF777FF00252846BDE8F08100BFE5
:1013E00030020020CE3900080B3A0008C839000846
:1013F00044020020E40C0020463A00087A3A000833
:10140000903A0008953A00082402002038B50D4BA8
:101410001C6824B10C4801F069F9012410E00B4D5F
:101420000B48296801F0F0F82A680A490A48FFF7D2
:1014300049FF4FF48072214606482C6001F030F8D5
:10144000204638BD300200209A3A0008DC0C00200B
:10145000C23A0008E40D0020903A000800B50748A1
:10146000A1B001F043F9064801F040F9054801F048
:101470003DF980226946044800F08EFAD63A000809
:10148000F63A0008423B0008203C00087047000084
:1014900070B505460C46FEF7D9FF2B6806462BB9FA
:1014A0004FF0FF332B60FEF7D9FF18E0CCB10F4BA4
:1014B0001C6802212046FEF7D9FE2B68013305D1B6
:1014C00004F108032B600023A36003E021462846B3
:1014D000FFF7E0F83046FEF7C1FFFEF781FF01207D
:1014E00070BDFEF7BBFF204670BD00BF200400208A
:1014F00070B50446FEF7AAFF256806461DB16B1CB1
:1015000005D100232360BDE87040FEF7A7BF284641
:101510000A2150F808392360FEF7A8FE236813B9A2
:101520004FF0FF33236015F8034C3046FEF796FF6B
:101530002046BDE87040FEF7D9BE0000104BD3F83E
:10154000882042F47002C3F888204FF000629A604D
:10155000102283F822200021DA7701F1604000F5A3
:1015600061400131522980F80023F6D11A6942F016
:1015700010021A615A6942F400725A61704700BF42
:1015800000ED00E08368DB0710B5044606D5C068AF
:10159000064BC0B253F821309847E060044B1B68FB
:1015A0001BB1BDE81040FFF75BB810BDE40E002092
:1015B000180400202DE9F0438BB070B1012874D1DC
:1015C0000D233C4A04930F210523019202920392BA
:1015D0000793059108930E220AE0374A01920523EA
:1015E0000721029203920493079305910893062220
:1015F0000692099300210327022601250F2404AA3D
:1016000001AB52F8212053F821304FEA420E1868FE
:1016100007FA0EF96FEA090C00EA0C001860D3F81B
:10162000008006FA0EF048EA0008C3F80080D3F8FC
:1016300008800CEA0808C3F80880D3F808E049EAF3
:101640000E0EC3F808E0D3F804E005FA02F82EEA1B
:10165000080EC3F804E0D3F80CE00CEA0E0EC3F851
:101660000CE0D3F80CE0072A40EA0E00D4BF4FF09C
:10167000000E4FF0010ED86003EB8E03A2EBCE02FA
:10168000186A920004FA02FE20EA0E000DF11C0E08
:1016900018625EF821E0186A0EFA02F20131024384
:1016A00003291A62ABD1002001E04FF0FF300BB0EC
:1016B000BDE8F0830004024000000240F8B5064691
:1016C0000F46042A04D8DFE802F05C060A0E120076
:1016D0004FF0FF30F8BD2C4B1C5C05340AE02A4B60
:1016E0001C5C043406E0284B1C5C023402E0264BF0
:1016F0001C5C0134E4B2A6B1012E42D14FF480410A
:101700000020FFF799FB02210846FFF795FB022115
:101710000846FFF791FB02210846FFF78DFB1B4DA2
:1017200011E04FF480510120FFF786FB01210220D8
:10173000FFF782FB01210220FFF77EFB012102203F
:10174000FFF77AFB124D3046FFF734FFEB690020BC
:1017500023F40063EB61286068602B6843F44073F6
:101760002B602B6843EAC4042C602B6843F004030D
:101770002B602968394329602B6843F040032B60B4
:10178000F8BD6FF00100F8BD5C3C00080038004077
:1017900000300140F8B50F4616460546C8B101288D
:1017A0004CD14FF480410020FFF746FB0221084650
:1017B000FFF742FB02210846FFF73EFB02210846E5
:1017C000FFF73AFB1F4B204C102283F824235A606A
:1017D00017E04FF480510120FFF72EFB012102207A
:1017E000FFF72AFB01210220FFF726FB012102203F
:1017F000FFF722FB134B154C102283F823230822FA
:101800005A602846FFF7D6FEE369002023F4006300
:10181000E36120606060636843F0400363602168B7
:1018200039432160236843F400732360084B43F875
:101830002560236843F040032360F8BD4FF0FF307C
:10184000F8BD00BF00E100E000380040003001407A
:10185000E40E0020012808B507D8054B012103EB51
:101860008000FFF715FE002008BD4FF0FF3008BDD7
:10187000EC0E0020012808B506D8054B03EB8000CC
:10188000FFF736FE002008BD4FF0FF3008BD00BF57
:10189000EC0E002018B101280ED1094B00E0094BD5
:1018A00098688007FCD5D9609968C907FCD5DB68C2
:1018B00002B11370012070474FF0FF30704700BF36
:1018C000003800400030014010B1012802D07047BC
:1018D000024B00E0024BD960704700BF003001406E
:1018E0000038004000210148FFF74CBE00300140A5
:1018F00001210148FFF746BE003800402DE9F341C1
:1019000006460D46174698460024444510D00DF172
:1019100007020DB1295D00E029463046FFF7BAFF06
:10192000002807DB17B19DF807303B550134ECE781
:10193000204601E04FF0FF3002B0BDE8F08100002A
:101940000C4B0146186882689368013B002B10B469
:10195000936005DA9469A34208DBCBB20A2B05D069
:101960001368581C1060197010BC704710BC00F050
:10197000E5BF00BFA802002008B53E20FFF7E0FF4A
:101980002020FFF7DDFF034B1B689868BDE8084087
:1019900000F068BCA80200202DE9804885B081468F
:1019A00000AF0E469246FFF7E7FFB0460AF1FF345C
:1019B0000025C6EB0803A342F5DA844B186841689A
:1019C0004B68013B002B4B6004DA00F097FE0028C7
:1019D00004DAE8E70B685A1C0A6018780D2801D071
:1019E0000A280FD100240D2088F80040FFF7A8FF37
:1019F0000A20FFF7A5FF4645D5D0334622462546A7
:101A000020462BE0082801D07F280DD14645D0D0B4
:101A1000082008F8015CFFF793FF2020FFF790FFF4
:101A200008F1FF3B082003E008F1010B88F80000F3
:101A3000FFF786FFD846BCE7222913D15C781CB398
:101A40005C2C25D001331C788C42F7D159782029A1
:101A50001AD80135197811B303F8010B1978202928
:101A6000F8D9E9E7272906D1E8E74B1C497822296C
:101A70000AD02029EDD91C785C2C1946F5D1591CC7
:101A80005B780132002BF0D1514800F02FFE8AE73D
:101A90009C1C9B780132002BF6D02346D3E7002D07
:101AA00081D0AB000E3323F00703EB46ADEB030D03
:101AB0006C464DF82510304690F800E003460130A2
:101AC000BEF1000FF8D0BEF1220F02D0BEF1270FF9
:101AD00000D1013344F821301846013390F800E07A
:101AE000BEF1000FF8D101318D42E5D1201FBAB10E
:101AF00050F8043FA3B1194613F801EBBEF1000FF3
:101B0000F5D0BEF15C0FF6D191F800E0BEF1000F08
:101B100004D091F801E001F801EBF5E7013AEAD1D0
:101B20002C4B2268FB60C7F80890002307F10801DE
:101B300051F82380B8F1000F0DD10133022B16D0DC
:101B4000F4E711463B607A6000F047FE7A683B6834
:101B500030B108F10C08D8F800000028F1D1ECE70A
:101B6000D8F808301BB12146284698472CE0216858
:101B7000194800F032FE054610BB184A18491948AA
:101B800000F042FD184800F0B1FD124BC7F8089074
:101B9000FB602C4607F1080353F824500DB10C35B7
:101BA00003E00134022CF5D10EE00C3555F8181C79
:101BB0000029F6D055F8142C0A4800F025FDF4E76A
:101BC00021680A4800F020FDDD46ECE6A80200206E
:101BD0005E3C0008F83C0008773C00087C3C0008AC
:101BE000883C0008903C00089A3C0008C23C000871
:101BF00008B5FEF719FC002008BD000080F0004089
:101C000002E000BF81F0004142001FBF5FEA4103D4
:101C100092EA030F7FEA226C7FEA236C6AD04FEAD4
:101C20001262D2EB1363C1BFD21841404840414019
:101C3000B8BF5B42192B88BF704710F0004F40F4CB
:101C4000000020F07F4018BF404211F0004F41F4E7
:101C5000000121F07F4118BF494292EA030F3FD0B3
:101C6000A2F1010241FA03FC10EB0C00C3F12003C6
:101C700001FA03F100F0004302D5494260EB400055
:101C8000B0F5000F13D3B0F1807F06D340084FEAC0
:101C9000310102F10102FE2A51D2B1F1004F40EBB5
:101CA000C25008BF20F0010040EA0300704749001D
:101CB00040EB000010F4000FA2F10102EDD1B0FAE8
:101CC00080FCACF1080CB2EB0C0200FA0CF0AABFDD
:101CD00000EBC25052421843BCBFD040184370477B
:101CE00092F0000F81F4000106BF80F40000013281
:101CF000013BB5E74FEA41037FEA226C18BF7FEA58
:101D0000236C21D092EA030F04D092F0000F08BF99
:101D10000846704790EA010F1CBF0020704712F080
:101D20007F4F04D1400028BF40F00040704712F1BF
:101D300000723CBF00F50000704700F0004343F024
:101D4000FE4040F4000070477FEA226216BF08465A
:101D50007FEA23630146420206BF5FEA412390EA1D
:101D6000010F40F4800070474FF0000304E000BF13
:101D700010F0004348BF40425FEA000C08BF7047C4
:101D800043F0964301464FF000001CE050EA010288
:101D900008BF70474FF000030AE000BF50EA01029D
:101DA00008BF704711F0004302D5404261EB41018A
:101DB0005FEA010C02BF84460146002043F0B643AF
:101DC00008BFA3F18053A3F50003BCFA8CF2083AD4
:101DD000A3EBC25310DB01FA02FC634400FA02FCDD
:101DE000C2F12002BCF1004F20FA02F243EB0200E4
:101DF00008BF20F00100704702F1200201FA02FC46
:101E0000C2F1200250EA4C0021FA02F243EB020038
:101E100008BF20EADC7070474FF0FF0C1CEAD0527C
:101E20001EBF1CEAD15392EA0C0F93EA0C0F6FD03D
:101E30001A4480EA010C400218BF5FEA41211ED01B
:101E40004FF0006343EA501043EA5111A0FB013107
:101E50000CF00040B1F5000F3EBF490041EAD371DC
:101E60005B0040EA010062F17F02FD2A1DD8B3F158
:101E7000004F40EBC25008BF20F00100704790F0C7
:101E8000000F0CF0004C08BF49024CEA502040EA19
:101E900051207F3AC2BFD2F1FF0340EAC2507047DF
:101EA00040F400004FF00003013A5DDC12F1190F1D
:101EB000DCBF00F000407047C2F10002410021FA8F
:101EC00002F1C2F1200200FA02FC5FEA310040F1A7
:101ED000000053EA4C0308BF20EADC70704792F020
:101EE000000F00F0004C02BF400010F4000F013A58
:101EF000F9D040EA0C0093F0000F01F0004C02BF53
:101F0000490011F4000F013BF9D041EA0C018FE7C1
:101F10000CEAD15392EA0C0F18BF93EA0C0F0AD0C7
:101F200030F0004C18BF31F0004CD8D180EA0100ED
:101F300000F00040704790F0000F17BF90F0004F86
:101F4000084691F0000F91F0004F14D092EA0C0F68
:101F500001D142020FD193EA0C0F03D14B0218BFFB
:101F6000084608D180EA010000F0004040F0FE4041
:101F700040F40000704740F0FE4040F440007047DD
:101F80004FF0FF0C1CEAD0521EBF1CEAD15392EA5C
:101F90000C0F93EA0C0F69D0A2EB030280EA010C4C
:101FA00049024FEA402037D04FF0805343EA1111E5
:101FB00043EA10130CF000408B4238BF5B0042F143
:101FC0007D024FF4000C8B4224BF5B1A40EA0C00E8
:101FD000B3EB510F24BFA3EB510340EA5C00B3EB1A
:101FE000910F24BFA3EB910340EA9C00B3EBD10F08
:101FF00024BFA3EBD10340EADC001B0118BF5FEA5A
:102000001C1CE0D1FD2A3FF650AF8B4240EBC25082
:1020100008BF20F0010070470CF0004C4CEA502043
:102020007F32C2BFD2F1FF0340EAC250704740F492
:1020300000004FF00003013A37E792F0000F00F084
:10204000004C02BF400010F4000F013AF9D040EA02
:102050000C0093F0000F01F0004C02BF490011F496
:10206000000F013BF9D041EA0C0195E70CEAD1538E
:1020700092EA0C0F08D142027FF47DAF93EA0C0F75
:102080007FF470AF084676E793EA0C0F04D14B0259
:102090003FF44CAF08466EE730F0004C18BF31F00B
:1020A000004CCAD130F000427FF45CAF31F0004305
:1020B0007FF43CAF5FE700BF42000ED2B2F1FE4FAB
:1020C0000BD34FF09E03B3EB126209D44FEA002307
:1020D00043F0004323FA02F070474FF000007047CE
:1020E00012F1610F01D1420202D14FF0FF3070476F
:1020F0004FF00000704700BF0A22002100F008BC2A
:102100008A892DE9F041054610070C4659D44B68E1
:10211000002B02DC0B6C002B17DDE66AAEB102F47B
:102120008052002392B22F682B600AB1606D15E0D7
:10213000216A01232846B047411C0FD12B686BB19F
:102140001D2B01D0162B03D12F600020BDE8F0819C
:10215000A38943F04003A381BDE8F081A3895A0716
:1021600005D56368C01A636B0BB1236CC01A0023DA
:102170000246E66A216A2846B047431CA38906D175
:1021800029681D293AD8214ACA40D60736D50022E7
:102190006260D9042269226004D5421C01D12B68F7
:1021A00003B96065616B2F600029CED004F1440350
:1021B000994202D0284600F07BF900206063BDE818
:1021C000F0810F69002FC0D093070E6808BF4B69DC
:1021D0000F6018BF0023C7EB06088B6002E00744BE
:1021E000C0EB0808B8F1000FAFDD43463A46216A5C
:1021F000A66A2846B0470028F1DCA38943F04003D3
:10220000A3814FF0FF30BDE8F08100BF0100402006
:1022100038B50B6905460C46DBB118B183690BB9BB
:1022200000F072F80C4B9C4201D16C6808E00B4B3B
:102230009C4201D1AC6803E0094B9C4208BFEC68AA
:10224000B4F90C302BB121462846BDE83840FFF7E1
:1022500057BF002038BD00BF103D0008303D0008CA
:10226000503D0008014620B9044B0549186800F0AC
:10227000D3B8044B1868FFF7CBBF00BF703D000810
:1022800011220008A8020020014900F0C5B800BFD3
:1022900011220008002310B50446036043608360E8
:1022A00081814366C28103614361836119460822CB
:1022B0005C3000F0F5F8054B6362054BA362054BFB
:1022C000E362054B2462236310BD00BF552700085D
:1022D00077270008AF270008D327000870B56823C8
:1022E0004D1E5D430E4605F1740100F02FF90446C2
:1022F00040B1002180E842000C30A06005F1680286
:1023000000F0CEF8204670BD836910B5044633BB9B
:102310008364C3640365124B124A1B68826298424D
:1023200004BF0123836100F01FF86060204600F0C5
:102330001BF8A060204600F017F80022E06004219E
:102340006068FFF7A7FF01220921A068FFF7A2FF3D
:1023500002221221E068FFF79DFF0123A36110BD57
:10236000703D000889220008F8B51C4B1E68B3694F
:10237000074613B93046FFF7C7FF4836B46873689D
:10238000013B04D4B4F90C507DB16834F8E73368EC
:102390000BB13668F2E704213846FFF79FFF306043
:1023A0000028F6D10C233B60F8BD4FF6FF73E381A4
:1023B0000123A38165662560A5606560256165616F
:1023C000A5610822294604F15C0000F069F8656304
:1023D000A563A564E5642046F8BD00BF703D000814
:1023E0002DE9F041884600F1480400268CB1A5682B
:1023F0006768013F0BD4AB89012B06D9B5F90E30C4
:10240000013302D02846C04706436835F1E7246807
:10241000ECE73046BDE8F0812DE9F8438046894677
:1024200000F14804002694B1A5686768013F0CD408
:10243000AB89012B07D9B5F90E30013303D02946FA
:102440004046C84706436835F0E72468EBE7304666
:10245000BDE8F88370B50E4B0E4CE41AA4100025AD
:102460001E46A54204D056F8253098470135F8E7B6
:10247000FDF78AFE084C094BE41AA41000251E46FD
:10248000A54204D056F8253098470135F8E770BDCD
:10249000B03E0008B03E0008B03E0008B03E000864
:1024A00002440346934202D003F8011BFAE7704747
:1024B00038B50546002946D051F8043C0C1F002BC6
:1024C000B8BFE41800F070FB1F4A1368114613B937
:1024D0006360146032E0A3420ED92268A0188342E0
:1024E00004BF18685B68636004BF121822600C6048
:1024F00024E0A24203D813465A68002AF9D118688A
:102500001918A1420BD12168014458188242196060
:1025100014D1106852685A60014419600EE002D963
:102520000C232B600AE021686018824204BF106807
:102530005268626004BF091821605C602846BDE8EB
:10254000384000F032BB38BDF80E002070B5CD1C0D
:1025500025F0030508350C2D38BF0C25002D064647
:1025600001DBA94202D90C23336046E000F01CFBDA
:10257000234B1C681A462146A1B10B685B1B0ED485
:102580000B2B03D90B60CC18CD501EE08C420DBF35
:1025900063684B686360136018BF0C4615E00C4617
:1025A0004968E9E7174C23681BB93046FDF7F0FD91
:1025B000206029463046FDF7EBFD431C18D0C41CB3
:1025C00024F00304A0420DD12560304600F0EDFA5E
:1025D00004F10B00231D20F00700C31A0ED05A424D
:1025E000E25070BD211A3046FDF7D2FD0130EBD12B
:1025F0000C233360304600F0D8FA002070BD00BFD5
:10260000F80E0020F40E00200FB40A4B13B51C681E
:1026100024B1A36913B92046FFF776FE05AB049AEF
:10262000A1680193204600F0E9FA02B0BDE810402D
:1026300004B07047A802002070B50E46054618B1D8
:1026400083690BB9FFF760FEAB69AC6813B9284624
:10265000FFF75AFE224B9C4201D16C6808E0214BE7
:102660009C4201D1AC6803E01F4B9C4208BFEC6860
:10267000A3891B0701D523693BB92146284600F0F1
:10268000B1F910B14FF0FF3070BD013EA36816F8EC
:10269000011F013BA36091B1002B04DAA2699342B0
:1026A00006DB0A2904D023685A1C22601970EDE762
:1026B0002246284600F042F90130E7D1E2E7002B3C
:1026C00008DA22460A21284600F038F90130D9D02C
:1026D0000A2070BD23680A205A1C2260187070BD41
:1026E000103D0008303D0008503D0008024B0146F7
:1026F0001868FFF7A1BF00BFA802002038B50C463C
:10270000054618B183690BB9FFF7FEFD0E4B9C42DD
:1027100001D16C6808E00D4B9C4201D1AC6803E02C
:102720000B4B9C4208BFEC682146284600F028FD70
:1027300038B96368013B636023685A1C22601878CB
:1027400038BD4FF0FF3038BD103D0008303D000867
:10275000503D000810B50C46B1F90E10FDF736FDDE
:102760000028ABBF636DA3891B1823F48053ACBF53
:102770006365A38110BD2DE9F0411F468B89DB0500
:1027800005460C46164605D502230022B1F90E1067
:10279000FDF729FDA389B4F90E1023F48053A3811A
:1027A00032463B462846BDE8F041FDF713BD10B563
:1027B0000C46B1F90E10FDF716FD431CA38915BF99
:1027C000606523F4805343F48053A38118BFA38131
:1027D00010BDB1F90E10FDF701BD10F8012B11F875
:1027E000013B012A28BF9A42F7D0D01A704703460E
:1027F00013F8012B002AFBD1181A013870472DE974
:10280000F0478046894692461E460F463D46089848
:1028100015F8014B00F054F92044427802F0080208
:1028200002F0FF030AB12F46F0E72D2C03D1BD1CA7
:102830007C78012303E02B2C04BF7C78BD1C16B1EF
:10284000102E0AD15EE0302C5AD12A7802F0DF0235
:10285000582A50D16C7810260235002B14BF4FF047
:1028600000426FF00042B2FBF6FE06FB1E21002282
:102870001046A4F13007092F01D83C460AE0A4F124
:102880004107192F01D8373C04E0A4F16107192F43
:1028900013D8573CA64210DD571C0BD0864507D3F2
:1028A00001D1A14203DB00FB0640012202E0704699
:1028B0004FF0FF3215F8014BDBE7511C0ED1002B16
:1028C0004FF0220314BF4FF000406FF00040C8F8F3
:1028D0000030BAF1000F07D1BDE8F08703B14042E4
:1028E000BAF1000F11D00AB1013D00E04D46CAF81F
:1028F0000050BDE8F0873024002EAED10826ACE7AA
:102900000A26AAE7302CA0D0A7E7BDE8F087000090
:10291000084B37B51C68084D236A002B08BF2B46AF
:10292000009313460A4601462046FFF768FF03B0AE
:1029300030BD00BFA8020020AC020020F8B50F4651
:102940001446054618B183690BB9FFF7DDFC224B2D
:102950009C4201D16C6808E0204B9C4201D1AC68DC
:1029600003E01F4B9C4208BFEC68A369A360A389E6
:102970001A0709D523693BB123682069181A6369CE
:102980009842FEB20FDB08E02146284600F02AF804
:102990000028F1D04FF0FF361BE021462846FFF714
:1029A00037FC0028F6D1A368013BA36023685A1CBA
:1029B00022601F7063690130984204D0A389DB074D
:1029C00007D50A2E05D121462846FFF721FC00280D
:1029D000E0D13046F8BD00BF103D0008303D000892
:1029E000503D0008324B70B51D6806460C4625B1B7
:1029F000AB6913B92846FFF787FC2E4B9C4201D1E7
:102A00006C6808E02C4B9C4201D1AC6803E02B4B76
:102A10009C4208BFEC68B4F90C309AB215071DD47B
:102A2000D00602D4092232603AE0510712D5616B18
:102A300041B104F14403994202D03046FFF738FD1A
:102A400000236363A38923F02403A381002363602D
:102A500023692360A38943F00803A38123694BB949
:102A6000A38903F42073B3F5007F03D021463046D9
:102A700000F04CF8A28912F0010305D00023A360F6
:102A800063695B42A36103E0920758BF6369A36077
:102A900023695BB9B4F90C3003F0800080B230B127
:102AA00043F04003A3814FF0FF3070BD002070BDA4
:102AB000A8020020103D0008303D0008503D0008ED
:102AC000D0F8EC00704770B50E46B1F90E10002931
:102AD00090B014461D4606DA00232B60B3891A060F
:102AE0000ED540230EE001AAFDF782FB0028F3DBA0
:102AF000029A02F47042A2F500535A425A412A60E7
:102B00004FF480630020236010B070BD8B8973B5D3
:102B10009E0705460C4610D401AB6A46FFF7D3FF6B
:102B2000009906462846FFF711FD68B9B4F90C3044
:102B30009A0522D443F00203A38104F147032360E2
:102B400023610123636118E00D4BAB62A389206010
:102B500043F08003A381009B6361019B20614BB123
:102B6000B4F90E102846FDF748FB18B1A38943F0CD
:102B70000103A381A0893043A08102B070BD00BFD2
:102B80008922000882B001B901A93AB143B1137892
:102B90000B601278101C18BF012003E0104601E002
:102BA0006FF0010002B07047704770479368013BB7
:102BB000002B10B4936008DA9469A34202DBCBB215
:102BC0000A2B02D110BCFFF7B9BE1368581C106065
:102BD0001970C8B210BC7047F8B506460F461446C7
:102BE000D518AC4208D03A4614F8011B3046FFF71E
:102BF000DDFF431CF5D100E00020F8BD2DE9F04FCA
:102C00009DB00C4617460393064618B183690BB96D
:102C1000FFF77AFB7F4B9C4201D1746808E07E4B42
:102C20009C4201D1B46803E07C4B9C4208BFF4682D
:102C3000A38918070CD5236953B1002309932023D6
:102C40008DF8293030238DF82A30DFF8D4B144E0F4
:102C500021463046FFF7C6FE0028EED04FF0FF3089
:102C6000D5E0039A111D12680391002A80F28C802E
:102C7000524243F002000792049098F800302E2B45
:102C800000F08480032298F80010654800F010FBE3
:102C900048B14023CBEB000003FA00F0049B18433B
:102CA000049008F1010898F800105E488DF828108B
:102CB000062208F1010700F0FBFA002800F09580D9
:102CC000594B002B40F08880039B073323F0070308
:102CD00008330393099B53440993B846454615F8B6
:102CE000013B1BB9B8EB07090FD003E0252BF9D046
:102CF000A846F3E74B463A4621463046FFF76CFFBD
:102D000001307FD0099B4B44099398F80030002B89
:102D100078D000234FF0FF32049307930592069377
:102D20008DF853301A930127052229783F4800F087
:102D3000BFFA05F10108049B38B13C4A801A07FA32
:102D400000F0184304904546EEE7D90644BF202220
:102D50008DF853201A0744BF2B228DF853202A7870
:102D60002A2A3FF47EAF079A00210A20A84601359F
:102D700098F80030303B092B03D800FB02320121C8
:102D8000F4E700293FF479AF079276E798F801302D
:102D90002A2B0BD1039B1A1D1B680392002BB8BF73
:102DA0004FF0FF3308F1020805936BE7002305930A
:102DB00008F1010019460A258046013098F80020E4
:102DC000303A092A03D805FB01210123F4E7002B3F
:102DD0003FF458AF059155E703AB00932246144BDF
:102DE00004A93046AFF3008007E003AB009322460E
:102DF0000F4B04A9304600F093F8B0F1FF3F824634
:102E00007FF468AFA3895B063FF528AF09981DB032
:102E1000BDE8F08F103D0008303D0008503D00082F
:102E2000823D0008863D0008000000007C3D00084F
:102E3000D92B00082DE9F04791461F460A698B6897
:102E4000DDF820809342B8BF1346C9F8003091F8EE
:102E5000432006460C4612B10133C9F800302368FE
:102E6000990642BFD9F800300233C9F8003025680E
:102E700015F0060510D104F1190A07E001235246A6
:102E800039463046C04701301AD00135E368D9F8D9
:102E900000209B1A9D42F1DB94F8433022680033F6
:102EA00018BF012392060FD5E1185A1C302081F873
:102EB0004300224494F8451082F84310023303E0A3
:102EC0004FF0FF30BDE8F08704F143023946304649
:102ED000C0470130F4D02268D9F80050E36802F00E
:102EE0000602042A08BF5D1B2269A3680CBF25EAFD
:102EF000E57500259342C4BF9B1AED184FF00009F9
:102F00001A344D4509D00123224639463046C04780
:102F10000130D5D009F10109F3E70020BDE8F087C1
:102F20002DE9F04317460A7E85B06E2A984606467C
:102F30000C460C9B01F1430E00F0AE8011D8632AC1
:102F400022D009D8002A00F0BB80582A40F0CA805D
:102F500081F84520834955E0642A1ED0692A1CD097
:102F6000C0E0732A00F0B08009D86F2A2ED0702AF2
:102F700040F0B8800A6842F020020A603EE0752AFC
:102F800024D0782A3AD0ADE01A6801F14205111D2B
:102F90001960136884F84230A8E021681A6811F0BB
:102FA000800F02D0111D196008E011F0400F02F1EE
:102FB0000401196002D0B2F9003000E01368002B60
:102FC0003CDA2D225B4284F8432037E021681A68FE
:102FD00011F0800F02D0111D196007E011F0400FB1
:102FE00002F10401196001D0138800E01368227E09
:102FF0005C496F2A14BF0A2208221BE078225A4932
:1030000084F845202268186812F0800F00F104054A
:103010001D6003D1550601D5038800E00368D00781
:1030200044BF42F0200222601BB9226822F0200235
:1030300022601022002084F8430001E049490A225E
:103040006568A560002D08DB206820F00400206082
:103050002BB9002D7DD175460CE0002B79D075463B
:10306000B3FBF2F002FB1033CB5C05F8013D0346E5
:103070000028F5D1082A0BD12368DA0708D523697F
:1030800062689A42DEBF302305F8013C05F1FF3546
:10309000C5EB0E0323612EE008681A68496910F039
:1030A000800F03D0101D1860136808E010F0400F67
:1030B00002F104001860136801D0198000E0196063
:1030C00000232361754616E01A68111D1960156802
:1030D00062680021284600F0EBF808B1401B6060F0
:1030E000636804E004F1420584F84220012323616F
:1030F000002384F84330CDF800803B4603AA2146E4
:103100003046FFF797FE013002D14FF0FF3026E046
:1031100023692A4639463046C0470130F5D0236836
:103120009B0710D5002504F1190907E001234A4641
:1031300039463046C0470130E7D00135E368039A8D
:103140009B1A9D42F2DBE068039B9842B8BF184689
:1031500005E00B7884F8423004F142058AE705B0B7
:10316000BDE8F0838D3D00089E3D0008838903F093
:103170000903092B01D1FFF775B800207047000043
:10318000F8B50C46054618B183690BB9FFF7BCF8D2
:103190003A4B9C4201D16C6808E0394B9C4201D10A
:1031A000AC6803E0374B9C4208BFEC68B4F90C20D4
:1031B0000023636093B29E065BD458071AD4D906E5
:1031C00005D4092342F040022B60A28151E01A0786
:1031D0000BD521462846FFF71BF8002849D1A389C3
:1031E000A06023F00803A381A061A38943F0040336
:1031F000A38110E0616B71B104F14403994202D0E4
:103200002846FFF755F9236C63600020606313B113
:10321000E36B2360F8BD23691BB921462846FFF7FD
:1032200075FCB4F90C70BEB2B3070FD00123A381B3
:10323000154B1649186806F00906FFF7D1F8092E54
:10324000A78103D121462846FEF75AFF2269226052
:10325000666A6369216A2846B047002860600BDC13
:10326000A38917BF002243F0200343F040036260AC
:10327000A3814FF0FF30F8BD0020F8BD103D0008DD
:10328000303D0008503D0008703D00086D310008D9
:1032900049B1FF2A85BF8A2303600A704FF0FF30CF
:1032A00098BF0120704708467047000000000000EA
:1032B00001F0FF01102A2BDB10F0070F08D010F8E7
:1032C000013B013A8B422DD010F0070F42B3F6D1EB
:1032D000F0B441EA012141EA014122F007047FF004
:1032E00000070023F0E80256083C85EA010586EA5B
:1032F000010685FA47F5A3FA87F586FA47F6A5FA97
:1033000087F68EB9EED1F0BC01F0FF0102F00702A2
:1033100032B110F8013B013A83EA010313B1F8D14D
:103320000020704701387047002D06BF354603382E
:10333000073815F0010F07D1013015F4807F02BF67
:10334000013015F4C03F0130F0BC0138704700BFB8
:103350004E4D492048414E444C455200484152444C
:10336000204641554C542048414E444C4552004D56
:10337000454D204D414E4147452048414E444C4526
:103380005200425553204641554C542048414E442A
:103390004C4552005553414745204641554C542019
:1033A00048414E444C4552004445425547204D4FFC
:1033B0004E2048414E444C45520044554D4D5920F5
:1033C00048414E444C4552002A2A2A2052494F5423
:1033D000206B65726E656C2070616E69633A0A25B8
:1033E000730A0A002A2A2A207265626F6F74696E56
:1033F000672E2E2E0A0A006D61696E28293A205424
:103400006869732069732052494F542120285665FA
:103410007273696F6E3A20323031372E30312D643D
:103420006576656C2D3234332D6739623331322D38
:1034300056616E64726973290A0069646C65006D77
:1034400061696E0000440040000002000300024079
:103450000200024007002606040000000048004069
:1034600000000400090C0240080C0240070027037A
:103470000400000048656C6C6F204D6173746572C8
:1034800021206162636465666768696A6B6C6D6E52
:103490006F707172737475767778797A2030313203
:1034A000333435363738392041424344454647485E
:1034B000494A4B4C4D4E4F50515253545556575804
:1034C000595A0075736167653A202573203C64651D
:1034D000763E203C637320706F72743E203C6373B1
:1034E0002070696E3E205B6D6F6465205B73706554
:1034F00065645D5D0A0020202020202020204445B6
:10350000562069732074686520535049206465769D
:1035100069636520746F207573653A002020202050
:103520002020202020202020202569202D205350DD
:10353000495F25690A002020202020202020637375
:1035400020706F72743A2020706F727420746F2034
:1035500075736520617320746865206368697020E5
:1035600073656C656374206C696E65002020202093
:103570002020202063732070696E3A20202070691B
:103580006E20746F20757365206F6E2074682067DD
:103590006976656E20706F7274206173206373208A
:1035A0006C696E650020202020202020206D6F6433
:1035B000653A206D757374206265206F6E65206FAB
:1035C000662074686520666F6C6C6F77696E672023
:1035D0006F7074696F6E7320282A206D61726B732F
:1035E0002064656661756C742076616C7565293A36
:1035F000002020202020202020202020202A3020D1
:103600002D20504F4C3A302C2050484153453A30F1
:10361000202D204F4E2046495253542052495349A1
:103620004E472045444745002020202020202020D0
:10363000202020202031202D20504F4C3A302C20AB
:1036400050484153453A31202D204F4E2053454399
:103650004F4E4420524953494E4720454447450068
:103660002020202020202020202020202032202D3B
:1036700020504F4C3A312C2050484153453A30208D
:103680002D204F4E2046495253542046414C4C4920
:103690004E47204544474500202020202020202060
:1036A000202020202033202D20504F4C3A312C2038
:1036B00050484153453A31202D206F6E2073656389
:1036C0006F6E642066616C6C696E67206564676507
:1036D00000202020202020202073706565643A207F
:1036E0006D757374206265206F6E65206F6620743F
:1036F000686520666F6C6C6F77696E67206F707499
:10370000696F6E7320286F6E6C7920757365642005
:10371000696E206D6173746572206D6F6465293AFE
:1037200000202020202020202020202020203020A9
:103730002D20313030204B487A00202020202020BE
:103740002020202020202031202D20343030204BFC
:10375000487A002020202020202020202020202AFD
:1037600032202D2031204D487A002020202020209A
:103770002020202020202033202D2035204D487A65
:103780000020202020202020202020202020342045
:103790002D203130204D487A0A006572726F723ADE
:1037A00020696E76616C6964204445562076616CB0
:1037B000756520676976656E006572726F723A2072
:1037C000696E76616C6964204D4F44452076616C6A
:1037D000756520676976656E006572726F723A2052
:1037E000696E76616C69642053504545442076616A
:1037F0006C756520676976656E007370695F696EC8
:1038000069745F6D61737465723A206572726F726C
:1038100020696E697469616C697A696E67205350BA
:10382000495F2569206465766963652028636F6454
:1038300065202569290A006770696F5F696E697480
:103840003A206572726F7220696E697469616C6981
:103850007A696E67204750494F5F50494E28256965
:103860002C20256929206173204353206C696E65E3
:103870002028636F6465202569290A005350495F39
:103880002569207375636365737366756C6C792045
:10389000696E697469616C697A6564206173206D11
:1038A00061737465722C2063733A204750494F5FEF
:1038B00050494E2825692C202569292C206D6F64DC
:1038C000653A2025692C2073706565643A20256966
:1038D0000A007370695F696E69745F736C61766505
:1038E0003A206572726F7220696E697469616C69E1
:1038F0007A696E67205350495F256920646576694F
:1039000063652028636F64653A202569290A00678A
:1039100070696F5F696E69745F696E743A20657271
:10392000726F7220696E697469616C697A696E6719
:10393000204750494F5F50494E2825692C20256962
:1039400029206173204353206C696E652028636FC2
:103950006465202569290A005350495F2569207351
:1039600075636365737366756C6C7920696E6974D1
:1039700069616C697A656420617320736C61766536
:103980002C2063733A204750494F5F50494E2825F9
:10399000692C202569292C206D6F64653A202569E2
:1039A0000A0025347300202025326920000A2020D7
:1039B000202000203078253032780020203F3F2022
:1039C000002020202563200048656C6C6F00657224
:1039D000726F723A206E6F6465206973206E6F7427
:1039E00020696E697469616C697A6564206173200D
:1039F0006D61737465722C20706C656173652064F1
:103A00006F20736F206669727374004E6F2064615B
:103A1000746120746F207472616E736665722067C2
:103A20006976656E2C2077696C6C207472616E7398
:103A3000666572202748656C6C6F2720746F206460
:103A40006576696365006572726F723A20756E61A2
:103A5000626C6520746F207472616E73666572208B
:103A60006461746120746F20736C617665202863D3
:103A70006F64653A202569290A005472616E736685
:103A8000657265642025692062797465733A0A005D
:103A90004D4F5349004D49534F006572726F723A52
:103AA000206E6F6465206973206E6F7420696E6983
:103AB0007469616C697A656420617320736C6176E6
:103AC00065005265636569766564202569206279C1
:103AD0007465733A0A000A52494F54206C6F772D6F
:103AE0006C6576656C205350492064726976657206
:103AF00020746573740054686973206170706C6918
:103B0000636174696F6E20656E61626C65732079A4
:103B10006F7520746F2074657374206120706C6100
:103B200074666F726D7320535049206472697665B4
:103B30007220696D706C656D656E746174696F6E0D
:103B40002E00456E746572202768656C702720749E
:103B50006F2067657420737461727465640A00690C
:103B60006E69745F6D617374657200496E69746922
:103B7000616C697A65206E6F6465206173205350B3
:103B800049206D617374657200696E69745F736C4E
:103B900061766500496E697469616C697A65206E49
:103BA0006F64652061732053504920736C617665A2
:103BB0000073656E64005472616E73666572207383
:103BC0007472696E6720746F20736C61766520284B
:103BD0006F6E6C7920696E206D6173746572206DF3
:103BE0006F646529007072696E745F72780050723C
:103BF000696E7420746865207265636569766564B2
:103C000020737472696E6720286F6E6C7920696EFC
:103C100020736C617665206D6F646529000000007B
:103C20005F3B00086B3B00084D110008893B000812
:103C3000943B000811120008B13B0008B63B000895
:103C400051130008E53B0008EE3B00080D14000886
:103C50000000000000000000000000000100736888
:103C6000656C6C3A20696E636F7272656374207163
:103C7000756F74696E670068656C70004465736386
:103C800072697074696F6E00436F6D6D616E640070
:103C9000252D3230732025730A002D2D2D2D2D2D2D
:103CA0002D2D2D2D2D2D2D2D2D2D2D2D2D2D2D2D44
:103CB0002D2D2D2D2D2D2D2D2D2D2D2D2D2D2D2D34
:103CC0002D007368656C6C3A20636F6D6D616E6476
:103CD000206E6F7420666F756E643A2025730A003B
:103CE0007265626F6F74005265626F6F74207468E2
:103CF00065206E6F64650000E03C0008E73C00084A
:103D0000F11B00080000000000000000000000009F
:103D100000000000000000000000000000000000A3
:103D20000000000000000000000000000000000093
:103D30000000000000000000000000000000000083
:103D40000000000000000000000000000000000073
:103D50000000000000000000000000000000000063
:103D60000000000000000000000000000000000053
:103D7000480200204300504F53495800232D302B58
:103D80002000686C4C00656667454647003031325C
:103D900033343536373839414243444546003031B3
:103DA0003233343536373839616263646566000012
:103DB00020202020202020202028282828282020DB
:103DC00020202020202020202020202020202020F3
:103DD000881010101010101010101010101010106B
:103DE000040404040404040404041010101010104B
:103DF0001041414141414101010101010101010124
:103E00000101010101010101010101101010101057
:103E100010424242424242020202020202020202F4
:103E2000020202020202020202020210101010201C
:103E30000000000000000000000000000000000082
:103E40000000000000000000000000000000000072
:103E50000000000000000000000000000000000062
:103E60000000000000000000000000000000000052
:103E70000000000000000000000000000000000042
:103E80000000000000000000000000000000000032
:103E90000000000000000000000000000000000022
:103EA0000000000000000000000000000000000012
:103EB000000F002000000000F0040020400000007F
:103EC00000000000000000003A3400083F34000801
:103ED000FF000000FFFFFFFFFFFFFFFFFF000000EC
:103EE000FFFFFFFFFFFFFFFFFFFFFFFFFF000000DF
:103EF000FFFFFFFFFFFFFFFF00000000103D000875
:103F0000303D0008503D00080000000000000000A7
:103F100000000000000000000000000000000000A1
:103F20000000000000000000000000000000000091
:103F30000000000000000000000000000000000081
:103F40000000000000000000000000000000000071
:103F500000000000000000004802002043000000B4
:103F60000000000000000000000000000000000051
:103F700000000000000000000000000043000000FE
:103F80000000000000000000000000000000000031
:103F900000000000000000000000000043000000DE
:103FA0000000000000000000000000000000000011
:103FB00000000000000000000000000043000000BE
:103FC00000000000000000000000000000000000F1
:103FD000000000000000000000000000430000009E
:103FE00000000000000000000000000000000000D1
:103FF000000000000000000000000000430000007E
:1040000000000000000000000000000000000000B0
:10401000000000000000000000000000430000005D
:104020000000000000000000000000000000000090
:1040300000000000000000000000000091320008B5
:10404000852B000800000000AF3D0008403B000841
:10405000F6330008F6330008F6330008F63300089C
:10406000F6330008F6330008F6330008F63300088C
:10407000F6330008FFFFFFFFFFFFFFFFFFFFFFFF1B
:10408000FFFF0000010041534349490000000000C8
:104090000000000000000000000000000000000020
:1040A00000000000000041534349490000000000A7
:1040B0000000000000000000000000000000000000
:0840C0000000000000000000F8
:04000005080004717A
:00000001FF
